:020000040000FA
:100000000C943C010C946D010C946D010C946D01E9
:100010000C946D010C946D010C946D010C946D01A8
:100020000C946D010C946D010C946D010C946D0198
:100030000C946D010C94B3080C946D010C946D013B
:100040000C946D010C946D010C946D010C946D0178
:100050000C946D010C946D010C946D010C94690865
:100060000C946D010C943D090C9413090C946D01D2
:100070000C946D010C946D010C946D010C946D0148
:100080000C946D010C946D010C946D010C946D0138
:100090000C946D010C946D010C946D010C946D0128
:1000A0000C946D010C946D010C946D010C946D0118
:1000B0000C946D010C946D010C946D010C946D0108
:1000C0000C946D010C946D010C946D010C946D01F8
:1000D0000C946D010C946D010C946D010C946D01E8
:1000E0000C946D010C945E030C94CE010C94C80129
:1000F0000C94AB030C9473090C949F010C94C802EC
:100100000C94C4010C94D2010C94A2010C94180319
:100110000C94AC010C9426030C949B010C948D015F
:100120000C94FC030C94BA010C9404030C94F50297
:100130000C9493010C94CD010C94A8010C943B08F1
:100140000C94C0010C94B2010C94B6010C9497016C
:100150000C9402040200002100240027002A002D34
:10016000003000330001010000040107010A010012
:10017000002200250028002B002E00310034000250
:10018000010000050108010B0100002000230026EA
:100190000029002C002F003200000100000301069E
:1001A00001090105050505070508080808020202FE
:1001B000020A0A0808040404040101010101010102
:1001C000010303030303030303040707070C0C0CD9
:1001D0000C0C0C0C0C0202020206060606060606B1
:1001E000060B0B0B0B0B0B0B0B010210202008084E
:1001F0001020401020408002010201080402010189
:100200000204081020408080402010080402018071
:1002100004020180402010080402010804020101C8
:1002200002040810204080010204081020408000D1
:10023000000A0B02090C0D0E080703040100000060
:1002400000000000000000000000000000000000AE
:10025000000000000000000000000012111000006B
:10026000000000000000000000000000000000008E
:10027000000000000000730911241FBECFEFD1E27F
:10028000DEBFCDBF00E00CBF12E0A0E0B2E0E4EBC7
:10029000F3E200E00BBF02C007900D92A433B10758
:1002A000D9F723E0A4E3B2E001C01D92AC3DB20750
:1002B000E1F711E0CCE3D1E000E006C021970109AD
:1002C000802FFE010E94A911CB33D10780E00807DF
:1002D000A9F70E946B0A0C94D8110C94000081506D
:1002E000823108F05AC0E82FF0E08827E558FE4F29
:1002F0008F4F0C94A9119B019F018D0193019701D0
:10030000CD01A201A801AC01B201B601BA01C00140
:10031000C401CD01C801CE01D201809180008F7748
:10032000809380000895809180008F7DF9CF809127
:100330008000877FF5CF84B58F7784BD089584B51D
:100340008F7DFBCF8091B0008F778093B0000895B0
:100350008091B0008F7DF9CF809190008F7780934E
:1003600090000895809190008F7DF9CF809190004A
:10037000877FF5CF8091A0008F778093A0000895AC
:100380008091A0008F7DF9CF8091A000877FF5CF6D
:10039000809120018F778093200108958091200122
:1003A0008F7DF9CF80912001877FF5CFCF93DF93A9
:1003B000282F30E0F901E15DFD4F8491F901E7510B
:1003C000FE4FD491F901ED55FE4FC491CC23A1F01D
:1003D00081110E946F01EC2FF0E0EE0FFF1FE75735
:1003E000FE4FA591B491EC91ED2381E090E009F4EA
:1003F00080E0DF91CF91089580E090E0FACF1F93E5
:10040000CF93DF93282F30E0F901E15DFD4F849118
:10041000F901E751FE4FD491F901ED55FE4FC4911A
:10042000CC23A9F0162F81110E946F01EC2FF0E070
:10043000EE0FFF1FE159FE4FA591B4918FB7F894CD
:10044000EC91111108C0D095DE23DC938FBFDF91B2
:10045000CF911F910895DE2BF8CFCF93DF9390E0DB
:10046000FC01E751FE4F24918D559E4FFC01849174
:100470008823D1F090E0880F991FFC01EB5AFE4FC2
:10048000A591B491FC01E159FE4FC591D491623020
:1004900071F49FB7F8943C91822F809583238C93BD
:1004A000E8812E2B28839FBFDF91CF9108958FB7CE
:1004B000F894EC912E2B2C938FBFF6CF3FB7F89486
:1004C0008091550290915602A0915702B091580226
:1004D00026B5A89B05C02F3F19F00196A11DB11D9F
:1004E0003FBFBA2FA92F982F8827BC01CD01620FDB
:1004F000711D811D911D42E0660F771F881F991F96
:100500004A95D1F708959091000289130DC0E4E552
:10051000F1E0E4919FEF90930002E230E1F038F4D3
:10052000EE2381F0E13089F060E00C94FF01E430CB
:1005300049F110F1E530C1F7909173009D7F9093E0
:100540007300F2CF10926E00EFCF90916F009D7FFD
:1005500090936F00E9CF909170009D7F9093700011
:1005600091E09093B0009091B100987F9460909347
:10057000B1001092B300D8CF909171009D7F9093FD
:100580007100D2CF909172009D7F90937200CCCF7A
:10059000AF92BF92CF92DF92EF92FF920F931F9391
:1005A000CF93DF936C017B018B01040F151FEB01CF
:1005B0005E01AE18BF08C017D10759F06991D60186
:1005C000ED91FC910190F081E02DC6011995892BE8
:1005D00079F7C501DF91CF911F910F91FF90EF90B7
:1005E000DF90CF90BF90AF900895FC01538D448D64
:1005F000252F30E0842F90E0821B930B541710F0CE
:10060000CF96089501970895FC01918D828D9817DA
:1006100061F0A28DAE0FBF2FB11D5D968C91928DB2
:100620009F5F9F73928F90E008958FEF9FEF0895E3
:10063000FC01918D828D981731F0828DE80FF11DAC
:10064000858D90E008958FEF9FEF0895FC01918DC7
:10065000228D892F90E0805C9F4F821B91098F73C0
:100660009927089589E592E00E94260321E0892BCD
:1006700009F420E0822F0895FC01A48DA80FB92F62
:10068000B11DA35ABF4F2C91848D90E001968F73BA
:100690009927848FA689B7892C93A089B1898C91D9
:1006A000837080648C93938D848D981306C0028828
:1006B000F389E02D80818F7D80830895EF92FF92F2
:1006C0000F931F93CF93DF93EC0181E0888F9B8D75
:1006D0008C8D98131AC0E889F989808185FF15C02F
:1006E0009FB7F894EE89FF896083E889F989808152
:1006F0008370806480839FBF81E090E0DF91CF9121
:100700001F910F91FF90EF900895F62E0B8D10E042
:100710000F5F1F4F0F731127E02E8C8D8E110CC0B1
:100720000FB607FCFACFE889F989808185FFF5CFFC
:10073000CE010E943C03F1CFEB8DEC0FFD2FF11D9C
:10074000E35AFF4FF0829FB7F8940B8FEA89FB8939
:1007500080818062CFCFCF93DF93EC01888D882397
:10076000B9F0AA89BB89E889F9898C9185FD03C014
:10077000808186FD0DC00FB607FCF7CF8C9185FFF9
:10078000F2CF808185FFEDCFCE010E943C03E9CFFF
:10079000DF91CF91089580E090E0892B29F00E94AD
:1007A000320381110E94000080E090E0892B49F023
:1007B00080E090E0892B29F00E94000081110E94C6
:1007C000000080E090E0892B49F080E090E0892BE8
:1007D00029F00E94000081110E94000080E090E05A
:1007E000892B49F080E090E0892B29F00E940000DD
:1007F00081110C940000089521E030E0FC01378B5A
:10080000268B089521E030E0FC0136A725A7089546
:100810002F923F924F925F926F927F928F929F9210
:10082000AF92BF92CF92DF92EF92FF920F931F93FE
:10083000CF93DF93EC01698D7A8D8B8D9C8DA9A46C
:10084000BAA40BA51CA5611571058105910509F4D4
:1008500080C00E940B102DA13EA14FA158A50E945F
:10086000C21020E034E244E759E40E94630F962E60
:10087000872E382E292ECD8CDE8CEF8CF8A049A047
:100880005AA06BA07CA0A3019201C701B6010E94EF
:10089000BD101816D4F4292D382D432D522DC30127
:1008A000B2010E94F20E2B013C019B01AC01C70179
:1008B000B6010E94BD10181614F026013701C201BE
:1008C000D30189A39AA3ABA3BCA349A05AA06BA050
:1008D0007CA0A3019201C701B6010E945E0F87FFB1
:1008E0001AC0292D382D432D522DC301B2010E946B
:1008F000F10E3B014C019B01AC01C701B6010E9406
:100900005E0F87FD02C036014701C301D40189A3F0
:100910009AA3ABA3BCA349A05AA06BA07CA020E0E3
:1009200030E0A901C301B2010E94BD1018160CF4F9
:10093000FCC277FA709477F87094A3019201B50124
:10094000C8010E945E0F18160CF4F7C2A3019201B1
:10095000DDC29A2C8B2C302E212E8DCF20E030E062
:10096000A901C701B6010E945E0F8111EFCF81E09E
:1009700090E09EA78DA719A21AA21BA21CA2198EF5
:100980001A8E1B8E1C8E03C3E4E5F1E0149117FD53
:100990005BC361E0802F0E942D02112319F01230F9
:1009A00009F0F1C1F12CE12C60E072E18AE790E0FE
:1009B000A70196010E948A1129013A01BA01A901F1
:1009C00041505109610971094F3F51056105710598
:1009D00009F00CF4BDC160E472E48FE090E0A7017F
:1009E00096010E948A11BA01A90141505109610979
:1009F0007109123009F069C182E04F3F510561056C
:100A0000710509F00CF463C060E970ED83E090E0DB
:100A1000A70196010E948A11BA01A901415051090A
:100A20006109710983E04F3F51056105710509F0C6
:100A30000CF44DC068E478EE81E090E0A7019601E7
:100A40000E948A11BA01A901415051096109710935
:100A500084E04F3F510561057105C9F1C4F164E2BD
:100A600074EF80E090E0A70196010E948A11BA011C
:100A7000A901415051096109710985E04F3F5105B4
:100A80006105710521F118F162E17AE780E090E0FB
:100A9000A70196010E948A11BA01A901415051098A
:100AA0006109710986E04F3F51056105710579F0D3
:100AB00070F0B301A2019AE0759567955795479537
:100AC0009A95D1F7415051096109710987E09091D8
:100AD000B100987F892B8093B100123009F4F5C1E1
:100AE0000CF0ECC1112309F43AC1113009F0ACC289
:100AF00078C100930002E4E5F1E01491812F1F3FDB
:100B000009F4A2C2123009F475C060F41123A1F1F6
:100B1000113009F44DC087FD97C261E0802F0E941B
:100B20002D023DCF143009F4AEC008F489C0153051
:100B300091F710922001109221018091210188608B
:100B40008093210180912101816080932101802F78
:100B500090E0FC01ED55FE4FE491F0E0EE0FFF1F39
:100B6000E159FE4F25913491FC01E751FE4FE4918C
:100B7000E093340215E00DCF14BC15BC84B582603F
:100B800084BD85B5816085BD802F90E0FC01ED5569
:100B9000FE4FE491F0E0EE0FFF1FE159FE4F25916B
:100BA0003491FC01E751FE4FE491E0933802F1CE1D
:100BB0001092800010928100809181008860809363
:100BC000810080918100816080938100802F90E07E
:100BD000FC01ED55FE4FE491F0E0EE0FFF1FE159EF
:100BE000FE4F25913491FC01E751FE4FE491E093D3
:100BF0003702CFCE1092B0001092B1008091B000B9
:100C000082608093B0008091B10081608093B100D8
:100C1000802F90E0FC01ED55FE4FE491F0E0EE0FE7
:100C2000FF1FE159FE4F2591349130934E022093DE
:100C30004D02FC01E751FE4FE491E0934F02A9CE33
:100C400010929000109291008091910088608093A2
:100C5000910080919100816080939100802F90E0BD
:100C6000FC01ED55FE4FE491F0E0EE0FFF1FE1595E
:100C7000FE4F25913491FC01E751FE4FE491E09342
:100C8000360213E086CE1092A0001092A10080914F
:100C9000A10088608093A1008091A1008160809371
:100CA000A100802F90E0FC01ED55FE4FE491F0E0B3
:100CB000EE0FFF1FE159FE4F25913491FC01E751E2
:100CC000FE4FE491E093350264CE4F3F510561053C
:100CD000710509F00CF455C068E478EE81E090E00D
:100CE000A70196010E948A11BA01A9014150510938
:100CF0006109710984E01111C1CE83E04F3F5105B4
:100D00006105710541F13CF162E17AE780E090E034
:100D1000A70196010E948A11BA01A9014150510907
:100D20006109710984E04F3F51056105710599F032
:100D300090F0B301A2018AE07595679557954795A4
:100D40008A95D1F7415051096109710985E003C0C5
:100D500081E01111BCCE95B5987F892B85BD47BD2B
:100D60008FEF9FEFDC018093490290934A02A0939A
:100D70004B02B0934C0280916E00826080936E00B3
:100D800063C182E0E6CFF12CE12C60E072E18AE7FA
:100D900090E0A70196010E948A11BA01A901415071
:100DA00051096109710991E04115510581E0680718
:100DB00071057CF068E478EE81E090E0A70196018F
:100DC0000E948A11BA01A9014150510961097109B2
:100DD00093E01130D9F480918100887F892B809332
:100DE000810050938900409388008FEF9FEFDC01D2
:100DF0008093450290934602A0934702B093480225
:100E000080916F00826080936F001EC11330D9F40F
:100E100080919100887F892B809391005093990055
:100E2000409398008FEF9FEFDC01809341029093F5
:100E30004202A0934302B093440280917100826009
:100E40008093710001C11430D9F48091A100887F92
:100E5000892B8093A1005093A9004093A8008FEFA5
:100E60009FEFDC0180933D0290933E02A0933F02EE
:100E7000B093400280917200826080937200E4C05F
:100E8000153009F02ACE80912101887F892B80932B
:100E9000210150932901409328018FEF9FEFDC013E
:100EA0008093390290933A02A0933B02B0933C02A4
:100EB00080917300826080937300C6C0143059F231
:100EC0000CF4ACCF153029F3BFC04093B3008FEFC3
:100ED0009FEFDC018093500290935102A093520245
:100EE000B093530280917000826080937000ACC018
:100EF000802F0E948302A8C09501A801C701B601F6
:100F00000E94BD1087FF31C0A701960160E074E226
:100F100084E799E40E94630F0E94DC0F698F7A8F47
:100F20008B8F9C8F82E090E030C09501A801C301B7
:100F3000B2010E94BD1087FF09CD20E030E0A90179
:100F4000C701B6010E94BD101816B4F22601370180
:100F500077FA709477F87094A3019201B501C801F3
:100F60000E945E0F18160CF4F9CC9501A80160E000
:100F700074E284E799E40E94630F0E94DC0F698F9A
:100F80007A8F8B8F9C8F83E090E09EA78DA78F85B3
:100F90008F3F61F0898D9A8DAB8DBC8DB695A795ED
:100FA00097958795898F9A8FAB8FBC8F898D9A8DF6
:100FB000AB8DBC8D892B8A2B8B2BC1F020E030E0D0
:100FC000A90169A17AA18BA19CA10E945E0F881F33
:100FD0008827881F11E018278A89811739F08989A5
:100FE0008F3F21F0612F0E94FF011A8B898C9A8C10
:100FF000AB8CBC8C0C8181149104A104B10409F464
:1010000077CFC501B4010E940B109B01AC0160E0D9
:1010100074E284E799E40E94630F6B017C0120E095
:1010200030E048EF51E40E94BD1087FD61CFC70159
:10103000B6010E94DC0F6B0180910002801709F459
:10104000A3CC8F3F09F455CD8D829E82AF82B886A6
:10105000DF91CF911F910F91FF90EF90DF90CF9094
:10106000BF90AF909F908F907F906F905F904F90C8
:101070003F902F9008951F93CF93DF93EC018DA5A0
:101080009EA5029771F4888911E0813009F410E07F
:10109000811739F08F858F3F21F0612F0E94FF016A
:1010A000188B29A13AA14BA15CA16D8D7E8D8F8DEE
:1010B00098A10E945E0F882331F0CE01DF91CF917D
:1010C0001F910C940804DF91CF911F9108950E9405
:1010D000D3111F920F920FB60F9211242F933F93AB
:1010E0008F939F93AF93BF938091F6029091F702F5
:1010F000A091F802B091F9023091540223E0230F3D
:101100002D3758F50196A11DB11D209354028093EF
:10111000F6029093F702A093F802B093F90280913F
:10112000550290915602A0915702B0915802019633
:10113000A11DB11D8093550290935602A0935702B2
:10114000B0935802BF91AF919F918F913F912F9192
:101150000F900FBE0F901F90189526E8230F029650
:10116000A11DB11DD2CF1F920F920FB60F92112465
:101170000BB60F922F933F934F935F936F937F9391
:101180008F939F93AF93BF93EF93FF938091500200
:1011900090915102A0915202B0915302892B8A2B57
:1011A0008B2BE1F190914F02E0914D02F0914E02B4
:1011B0008081892780838091500290915102A09173
:1011C0005202B0915302181619061A061B069CF417
:1011D0008091500290915102A0915202B09153021D
:1011E0000197A109B1098093500290935102A093F5
:1011F0005202B0935302FF91EF91BF91AF919F9133
:101200008F917F916F915F914F913F912F910F90AF
:101210000BBE0F900FBE0F901F901895809100028B
:101220000E948302E8CF1F920F920FB60F921124F3
:101230000BB60F922F933F934F935F936F937F93D0
:101240008F939F93AF93BF93EF93FF9389E592E0C2
:101250000E943C03FF91EF91BF91AF919F918F91BD
:101260007F916F915F914F913F912F910F900BBEA6
:101270000F900FBE0F901F9018951F920F920FB6F0
:101280000F9211240BB60F922F938F939F93EF938E
:10129000FF93E0916902F0916A028081E0916F0210
:1012A000F091700282FD1DC09081809172028F5F6B
:1012B0008F7320917302821741F0E0917202F0E087
:1012C000E75AFD4F958F80937202FF91EF919F91A6
:1012D0008F912F910F900BBE0F900FBE0F901F900C
:1012E00018958081F2CF10925C0210925B0288EE1A
:1012F00093E0A0E0B0E080935D0290935E02A09343
:101300005F02B093600287E192E090935A0280936B
:10131000590285EC90E0909366028093650284EC1C
:1013200090E0909368028093670280EC90E0909345
:101330006A028093690281EC90E090936C02809342
:101340006B0282EC90E090936E0280936D0286ECCB
:1013500090E09093700280936F021092720210924C
:1013600073021092740210927502E1E3F3E080E0E0
:1013700090E0A8E4B3E440E050E068EC71E410824F
:101380001182828B938BA48BB58B46875787608B9A
:10139000718B15AA16AA17AA10AE82839383A48311
:1013A000B58386839783A087B18711AA12AA13AA4F
:1013B00014AAF99623E0EC3DF20709F782E093E0E6
:1013C00090930503809304038FEF8093060310929C
:1013D0000703109208031092090310920A03109257
:1013E0000B0310920C0310920D0310920E0329E1CF
:1013F00033E03093100320930F038093110392E0A6
:101400009093120380931303909314038093150316
:101410009093160381E08093170380931803109232
:101420001B0310921C0310921D0310921E031092B6
:101430001F03109220031092210310922203109296
:10144000230310922403109225031092260380E0B8
:1014500090E0AAE7B4E48093270390932803A09335
:101460002903B0932A0382E79BEFACEFB1E48093AA
:101470002B0390932C03A0932D03B0932E03109273
:10148000300310922F0389E292E09093030380933C
:10149000020381E392E090931A03809319032FB71C
:1014A000F8948091F6029091F702A091F802B09121
:1014B000F9022FBF8093FA029093FB02A093FC02E3
:1014C000B093FD021092FE021092FF0210920003F0
:1014D000109201030895789484B5826084BD84B528
:1014E000816084BD85B5826085BD85B5816085BD1F
:1014F00080916E00816080936E00109281008091D7
:10150000810082608093810080918100816080935E
:101510008100809180008160809380008091B10083
:1015200084608093B1008091B00081608093B000AE
:101530008091910082608093910080919100816000
:1015400080939100809190008160809390008091C1
:10155000A10082608093A1008091A10081608093AE
:10156000A1008091A00081608093A0008091210162
:10157000826080932101809121018160809321010B
:101580008091200181608093200180917A008460A5
:1015900080937A0080917A00826080937A008091B3
:1015A0007A00816080937A0080917A0080688093CD
:1015B0007A001092C100E0916902F0916A0282E023
:1015C0008083E0916502F09166021082E0916702EB
:1015D000F091680280E1808310927102E0916D02C7
:1015E000F0916E0286E08083E0916B02F0916C02D4
:1015F000808180618083E0916B02F0916C02808138
:1016000088608083E0916B02F0916C028081806839
:101610008083E0916B02F0916C0280818F7D8083EA
:1016200062E083E00E942D0262E082E00E942D02CF
:101630000DE012E067E0E62E62E0F62EC1E0D2E0B7
:1016400073E1672E72E0772E6E0157014801D401D5
:101650008C91B2E08B0E911C61E00E942D02F5018D
:101660008081F2E0AF0EB11C61E00E942D02D60134
:101670005C90B2E0CB0ED11C61E0852D0E942D0262
:1016800061E0852D0E94FF016814790401F731E3C0
:10169000C32E33E0D32E47E0642E42E0742E812C1B
:1016A000912C58E4A52E53E4B52E8881229660E053
:1016B0000E94FF01F7019081F2E0EF0EF11CD801CA
:1016C0008C910E5F1F4FF6018083918361E00E9431
:1016D0002D0260E0D6018C910E94FF0161E0F601CD
:1016E00081810E942D0260E0D60111968C910E94AA
:1016F000FF01F601828A938AA48AB58AF9E3CF0EA4
:10170000D11C6C167D0689F661E086E30E942D02ED
:1017100061E086E30E942D0286E38093060361E088
:101720008FEF0E942D028FEF80931103C2E0C093D0
:10173000120361E087E30E942D0287E38093130385
:10174000C093140380910F0390911003DC01ED917D
:10175000FC910190F081E02D199580E896E9A8E1CF
:10176000BBE48093270390932803A0932903B093AD
:101770002A0381E794EAA5E4B5E480932B039093D0
:101780002C03A0932D03B0932E0361E086E20E9408
:101790002D02C0903F03D0904003E0904103F090B1
:1017A000420320E030E04AEF54E4C701B6010E9452
:1017B000C2104B015C018092370390923803A092D3
:1017C0003903B0923A0380E090E4ACE1B6E4809350
:1017D000330390933403A0933503B093360320E092
:1017E00030E04AE754E4C701B6010E94C2106B0121
:1017F0007C0120E030E0A9010E94BD1020E030E033
:1018000040E05FE387FDE7C1C701B6010E94F20E29
:101810000E94D50F6B017C01C0923B03D0923C0328
:10182000E0923D03F0923E03A5019401C501B4018D
:101830000E94F20E4B015C010E9435119B01AC012C
:1018400060E074E284E799E40E94630F60935203BE
:1018500070935303809354039093550380E090E07A
:10186000A8ECB2E48093480390934903A0934A0301
:10187000B0934B03A501940160E27CEB8EEB9CE4FA
:101880000E94630F4B015C0120E030E0A9010E943F
:10189000BD1020E030E040E05FE387FDA1C1C5015D
:1018A000B4010E94F20E0E94D50F60934C03709316
:1018B0004D0380934E0390934F0380916603909164
:1018C0006703A0916803B0916903C81AD90AEA0AAC
:1018D000FB0A80913203F7FE88C1F094E094D09423
:1018E000C094C11CD11CE11CF11C2FEF3FEF3093C1
:1018F00051032093500361E00E94FF0180914C034B
:1019000090914D03A0914E03B0914F03880F991F02
:10191000AA1FBB1F8C159D05AE05BF0564F0F5948D
:10192000E794D794C794C0924C03D0924D03E092B1
:101930004E03F0924F038091520390915303A09174
:101940005403B09155038093560390935703A0938B
:101950005803B093590325EA34ED48E653E5609106
:101960003703709138038091390390913A030E94B4
:10197000630F60935E0370935F03809360039093A3
:10198000610381E080934703C3E0D0E040916603A8
:1019900050916703609168037091690380913B03E4
:1019A00090913C03A0913D03B0913E034817590725
:1019B0006A077B0709F421C180914703882361F0FE
:1019C0000E945E0260935A0370935B0380935C03F2
:1019D00090935D03109247030E945E026B017C01AD
:1019E00080915A0390915B03A0915C03B0915D03D9
:1019F00046015701881A990AAA0ABB0A6091560340
:101A00007091570380915803909159030E94DC0F05
:101A100086169706A806B90608F4B8CF80913B034E
:101A200090913C03A0913D03B0913E034091660329
:101A3000509167036091680370916903841B950B53
:101A4000A60BB70BB7FF07C0B095A09590958195F1
:101A50009F4FAF4FBF4F40914C0350914D0360914A
:101A60004E0370914F0384179507A607B70789F4B3
:101A700080915E0390915F03A0916003B091610338
:101A8000B05880935E0390935F03A0936003B0937C
:101A9000610361E0809131030E94FF01CE01019753
:101AA000F1F78091500390915103092E000CAA0B7D
:101AB000BB0B40916603509167036091680370917E
:101AC0006903840F951FA61FB71F80936603909329
:101AD0006703A0936803B0936903809056039090C6
:101AE0005703A0905803B0905903809262039092DC
:101AF0006303A0926403B092650320915E0330916A
:101B00005F034091600350916103C501B4010E94DD
:101B1000C210A50194010E94C2109B01AC0160E0BB
:101B200070E080E89FE30E94F10EA50194010E94FD
:101B3000C210609356037093570380935803909399
:101B4000590360E0809131030E94FF0180904803B7
:101B500090904903A0904A03B0904B03A5019401D3
:101B600060915603709157038091580390915903E7
:101B70000E945E0F87FF08C0809256039092570321
:101B8000A0925803B0925903C0925A03D0925B03BB
:101B9000E0925C03F0925D0340916603509167030D
:101BA000609168037091690380913B0390913C03BD
:101BB000A0913D03B0913E03481759076A077B0780
:101BC00009F0E4CE10926203109263031092640352
:101BD00010926503DBCEC701B6010E94F10E18CE4C
:101BE000C501B4010E94F10E5ECE21E030E03093D9
:101BF00051032093500360E07FCE8FB7F894C090DC
:101C0000F602D090F702E090F802F090F9028FBF50
:101C10008091FA029091FB02A091FC02B091FD022A
:101C2000A7019601281B390B4A0B5B0BCA01B901AE
:101C30000E940B1020E030E04AE754E40E94630F5A
:101C40006093FE027093FF02809300039093010360
:101C5000C092FA02D092FB02E092FC02F092FD02E6
:101C60008091070390910803A0910903B0910A03A2
:101C7000892B8A2B8B2B91F10E945E026B017C01D8
:101C800080910B0390910C03A0910D03B0910E0372
:101C9000B701A601481B590B6A0B7B0B8091070308
:101CA00090910803A0910903B0910A0348175907BE
:101CB0006A077B0798F08091040390910503DC018B
:101CC000ED91FC910190F081E02D1995C0920B03EC
:101CD000D0920C03E0920D03F0920E0383E00E9479
:101CE000D601EC0182E00E94D601CD2B09F058C04C
:101CF00020E030E04AE756E460911F037091200332
:101D000080912103909122030E945E0F8823B1F0FD
:101D100080E090E0AAE7B6E480931F03909320034D
:101D2000A0932103B093220380912F03909130035D
:101D3000892B21F082E093E00E94080489E592E07B
:101D40000E9426031816190624F489E592E00E94E1
:101D5000AB030E945E026B017C018AE0882E912C0D
:101D6000A12CB12C0E945E026C197D098E099F097D
:101D7000683E734081059105A8F3B1E08B1A910884
:101D8000A108B108E8EECE0EE3E0DE1EE11CF11C76
:101D900081149104A104B10429F70E94CB032DCF33
:101DA000892BB1F420E030E04AE756EC60911F0344
:101DB0007091200380912103909122030E945E0F75
:101DC000882309F4BBCF80E090E0AAE7B6ECA4CF6B
:101DD00010921F03109220031092210310922203ED
:101DE000ADCF5058BB27AA270E94090F0C9483102F
:101DF0000E94751038F00E947C1020F039F49F3F4B
:101E000019F426F40C9472100EF4E095E7FB0C9490
:101E10006C10E92F0E94941058F3BA1762077307E9
:101E20008407950720F079F4A6F50C94B6100EF40B
:101E3000E0950B2EBA2FA02D0B01B90190010C01DA
:101E4000CA01A0011124FF27591B99F0593F50F4F2
:101E5000503E68F11A16F040A22F232F342F44274A
:101E6000585FF3CF469537952795A795F040539542
:101E7000C9F77EF41F16BA0B620B730B840BBAF012
:101E80009150A1F0FF0FBB1F661F771F881FC2F77D
:101E90000EC0BA0F621F731F841F48F48795779591
:101EA0006795B795F7959E3F08F0B0CF9395880F4B
:101EB00008F09927EE0F9795879508950E9448108E
:101EC00008F481E008950E94770F0C9483100E941B
:101ED0007C1058F00E94751040F029F45F3F29F003
:101EE0000C946C1051110C94B7100C9472100E9449
:101EF000941068F39923B1F3552391F3951B550B77
:101F0000BB27AA2762177307840738F09F5F5F4FCC
:101F1000220F331F441FAA1FA9F335D00E2E3AF00B
:101F2000E0E832D091505040E695001CCAF72BD023
:101F3000FE2F29D0660F771F881FBB1F2617370774
:101F40004807AB07B0E809F0BB0B802DBF01FF27A6
:101F500093585F4F3AF09E3F510578F00C946C1007
:101F60000C94B7105F3FE4F3983ED4F386957795D1
:101F70006795B795F7959F5FC9F7880F911D96955F
:101F8000879597F90895E1E0660F771F881FBB1FBB
:101F9000621773078407BA0720F0621B730B840B68
:101FA000BA0BEE1F88F7E09508950E94DC0F689445
:101FB000B1110C94B71008950E949C1088F09F579F
:101FC00098F0B92F9927B751B0F0E1F0660F771F5D
:101FD000881F991F1AF0BA95C9F714C0B13091F053
:101FE0000E94B610B1E008950C94B610672F782FB8
:101FF0008827B85F39F0B93FCCF386957795679518
:10200000B395D9F73EF490958095709561957F4F83
:102010008F4F9F4F0895E89409C097FB3EF4909529
:102020008095709561957F4F8F4F9F4F9923A9F0B1
:10203000F92F96E9BB279395F69587957795679540
:10204000B795F111F8CFFAF4BB0F11F460FF1BC084
:102050006F5F7F4F8F4F9F4F16C0882311F096E917
:1020600011C0772321F09EE8872F762F05C06623C5
:1020700071F096E8862F70E060E02AF09A95660F7E
:10208000771F881FDAF7880F9695879597F9089537
:10209000990F0008550FAA0BE0E8FEEF1616170679
:1020A000E807F907C0F012161306E407F50798F0E1
:1020B000621B730B840B950B39F40A2661F0232BFA
:1020C000242B252B21F408950A2609F4A140A69576
:1020D0008FEF811D811D089597F99F6780E870E05B
:1020E00060E008959FEF80EC089500240A9416168E
:1020F000170618060906089500240A9412161306F6
:10210000140605060895092E0394000C11F4882383
:1021100052F0BB0F40F4BF2B11F460FF04C06F5F9F
:102120007F4F8F4F9F4F089557FD9058440F551F75
:1021300059F05F3F71F04795880F97FB991F61F049
:102140009F3F79F087950895121613061406551FC0
:10215000F2CF4695F1DF08C0161617061806991F2C
:10216000F1CF86957105610508940895E894BB2721
:1021700066277727CB0197F908950E94481008F445
:102180008FEF08950E94D5100C9483100E94751053
:1021900038F00E947C1020F0952311F00C946C1004
:1021A0000C94721011240C94B7100E94941070F3C8
:1021B000959FC1F3950F50E0551F629FF001729FEC
:1021C000BB27F00DB11D639FAA27F00DB11DAA1FFB
:1021D000649F6627B00DA11D661F829F2227B00D48
:1021E000A11D621F739FB00DA11D621F839FA00DD3
:1021F000611D221F749F3327A00D611D231F849F23
:10220000600D211D822F762F6A2F11249F57504079
:102210009AF0F1F088234AF0EE0FFF1FBB1F661FF4
:10222000771F881F91505040A9F79E3F510580F0BD
:102230000C946C100C94B7105F3FE4F3983ED4F309
:10224000869577956795B795F795E7959F5FC1F761
:10225000FE2B880F911D9695879597F9089519F48F
:1022600016F40C9472100C9475110E949C10B8F323
:102270009923C9F3B6F39F57550B87FF0E9483112B
:102280000024A0E640EA900180585695979528F4DE
:10229000805C660F771F881F20F0261737074807D6
:1022A00030F4621B730B840B202931294A2BA6952D
:1022B00017940794202531254A2758F7660F771F72
:1022C000881F20F026173707480730F4620B730B7E
:1022D000840B200D311D411DA09581F7B901842F7C
:1022E0009158880F9695879508959F3F31F09150AA
:1022F00020F4879577956795B795880F911D9695EA
:10230000879597F9089591505040660F771F881F61
:10231000D2F70895052E97FB1EF400940E94A11198
:1023200057FD07D00E94B11107FC03D04EF40C9466
:10233000A11150954095309521953F4F4F4F5F4FDC
:10234000089590958095709561957F4F8F4F9F4F21
:102350000895EE0FFF1F881F8BBF0790F691E02DA9
:102360001994A1E21A2EAA1BBB1BFD010DC0AA1FC6
:10237000BB1FEE1FFF1FA217B307E407F50720F0EE
:10238000A21BB30BE40BF50B661F771F881F991F69
:102390001A9469F760957095809590959B01AC01B2
:1023A000BD01CF01089581E090E0F8940C94D8111C
:1023B000F894FFCFFF3800180000003D001C00001B
:1023C000003C001A000000000000005E03C802F597
:1023D00002AB03260304031803000000003B0802BD
:0823E00004E9FF0000FC03000A
:020000040003F7
:10E000000D9489F10D94B2F10D94B2F10D94B2F129
:10E010000D94B2F10D94B2F10D94B2F10D94B2F1F0
:10E020000D94B2F10D94B2F10D94B2F10D94B2F1E0
:10E030000D94B2F10D94B2F10D94B2F10D94B2F1D0
:10E040000D94B2F10D94B2F10D94B2F10D94B2F1C0
:10E050000D94B2F10D94B2F10D94B2F10D94B2F1B0
:10E060000D94B2F10D94B2F10D94B2F10D94B2F1A0
:10E070000D94B2F10D94B2F10D94B2F10D94B2F190
:10E080000D94B2F10D94B2F10D94B2F10D94B2F180
:10E090000D94B2F10D94B2F10D94B2F10D94B2F170
:10E0A0000D94B2F10D94B2F10D94B2F10D94B2F160
:10E0B0000D94B2F10D94B2F10D94B2F10D94B2F150
:10E0C0000D94B2F10D94B2F10D94B2F10D94B2F140
:10E0D0000D94B2F10D94B2F10D94B2F10D94B2F130
:10E0E0000D94B2F141546D656761323536300041AF
:10E0F000726475696E6F206578706C6F72657220DE
:10E1000073746B3530305632206279204D4C530099
:10E11000426F6F746C6F616465723E004875683F52
:10E1200000436F6D70696C6564206F6E203D200048
:10E130004350552054797065202020203D20005FF9
:10E140005F4156525F415243485F5F3D2000415658
:10E1500052204C696243205665723D20004743437C
:10E160002056657273696F6E203D20004350552024
:10E1700049442020202020203D20004C6F7720663D
:10E18000757365202020203D20004869676820665F
:10E190007573652020203D200045787420667573D6
:10E1A00065202020203D20004C6F636B2066757336
:10E1B000652020203D20004D617220203720323024
:10E1C000313300312E362E3800342E332E350056A2
:10E1D00023202020414444522020206F7020636F70
:10E1E00064652020202020696E73747275637469E1
:10E1F0006F6E2061646472202020496E74657272B3
:10E20000757074006E6F20766563746F7200726A49
:10E210006D702020006A6D70200057686174207056
:10E220006F72743A00506F7274206E6F7420737541
:10E2300070706F72746564004D7573742062652030
:10E2400061206C6574746572002000577269747483
:10E25000696E672045450052656164696E672045B7
:10E26000450045452065727220636E743D00504F35
:10E27000525400303D5A65726F2061646472003FF1
:10E280003D43505520737461747300403D454550C3
:10E29000524F4D207465737400423D426C696E6B41
:10E2A000204C454400453D44756D70204545505215
:10E2B0004F4D00463D44756D7020464C415348001B
:10E2C000483D48656C70004C3D4C69737420492F83
:10E2D0004F20506F72747300513D51756974005234
:10E2E0003D44756D702052414D00563D73686F7707
:10E2F00020696E7465727275707420566563746FF0
:10E30000727300593D506F727420626C696E6B00BD
:10E310002A0011241FBECFEFD1E2DEBFCDBF01E046
:10E320000CBF12E0A0E0B2E0EEE1FDEF03E00BBFB6
:10E3300002C007900D92A030B107D9F712E0A0E01B
:10E34000B2E001C01D92AE30B107E1F70F9460F367
:10E350000D948DFE01E20EBF0FEF0DBF11241FBE05
:10E360000D9460F30D9400F020E030E040ED57E0B4
:10E3700005C0FA013197F1F72F5F3F4F2817390792
:10E38000C0F308959C01260F311DC901A0E0B0E043
:10E390002F5F3F4FABBFFC018791882361F08093D3
:10E3A000C6008091C00086FFFCCF8091C0008064D1
:10E3B0008093C000EACF08958DE08093C6008091DD
:10E3C000C00086FFFCCF8091C00080648093C000B5
:10E3D0008AE08093C6008091C00086FFFCCF8091C8
:10E3E000C00080648093C00008950F94C2F10F9420
:10E3F000DCF10895FC019081992359F09093C600B7
:10E400008091C00086FFFCCF8091C0008064809323
:10E41000C0003196992379F70895282F982F929567
:10E420009F70892F805D8A3308F0895F8093C600D2
:10E430008091C00086FFFCCF8091C00080648093F3
:10E44000C000822F8F70982F905D9A3308F0995FEB
:10E450009093C6008091C00086FFFCCF8091C000E1
:10E4600080648093C00008959C01FB01853691056E
:10E470001CF46330710594F0C90164E670E00F94F8
:10E480002EFE605D7F4F6093C6008091C00086FFC6
:10E49000FCCF8091C00080648093C0002B30310598
:10E4A00014F43297B4F0C90164E670E00F942EFEC4
:10E4B0006AE070E00F942EFE605D7F4F6093C600AF
:10E4C0008091C00086FFFCCF8091C0008064809363
:10E4D000C000C9016AE070E00F942EFEC0968093E0
:10E4E000C6008091C00086FFFCCF8091C000806490
:10E4F0008093C00008951F93182F8EE692EE60E07F
:10E500000F94C2F11093C6008091C00086FFFCCF2B
:10E510008091C00080648093C0000F94DCF11F9153
:10E5200008952F923F924F925F926F927F928F92B7
:10E530009F92AF92BF92CF92DF92EF92FF920F9392
:10E540001F93DF93CF93CDB7DEB762970FB6F894E2
:10E55000DEBF0FBECDBF382E622ECA01DB015C01CB
:10E560006D01772420E2222E2E010894411C511CBB
:10E570008BC081E0A81680E0B80681E0C80680E084
:10E58000D80628F0C601AA27BB270F940DF2BB2797
:10E59000AD2D9C2D8B2D0F940DF28A2D0F940DF225
:10E5A0002092C6008091C00086FFFCCF8091C00001
:10E5B00080648093C0009DE29093C6008091C0006B
:10E5C00086FFFCCF8091C00080648093C0002092C1
:10E5D000C6008091C00086FFFCCF8091C00080649F
:10E5E0008093C00019828601750188249924A1E0D6
:10E5F0003A1651F03A1620F0B2E03B1661F409C029
:10E600000BBFF701779007C0C7010F9477FE782EF4
:10E6100002C0F7017080872D0F940DF22092C60082
:10E620008091C00086FFFCCF8091C0008064809301
:10E63000C000872D8052F401EF70F0708F3520F408
:10E64000E40DF51D708204C0E40DF51D8EE280839B
:10E650000894E11CF11C011D111D0894811C911CE2
:10E6600090E18916910409F0C2CF80E190E0A0E02A
:10E67000B0E0A80EB91ECA1EDB1E198AC2010F9493
:10E68000FAF10F94DCF16A94662009F072CF629679
:10E690000FB6F894DEBF0FBECDBFCF91DF911F91B3
:10E6A0000F91FF90EF90DF90CF90BF90AF909F9031
:10E6B0008F907F906F905F904F903F902F90089534
:10E6C0002F923F924F925F926F927F928F929F9282
:10E6D000AF92BF92CF92DF92EF92FF920F931F9370
:10E6E000DF93CF93CDB7DEB7CD53D1400FB6F894BB
:10E6F000DEBF0FBECDBF01E20EBF0FEF0DBF94B75F
:10E70000F894A89514BE80916000886180936000A1
:10E7100010926000789493FF05C0E0910002F091A0
:10E7200001021995279A2F9A8091C00082608093E8
:10E73000C00080E18093C40088E18093C1000000A4
:10E74000EE24FF24870144E0A42EB12CCC24DD2448
:10E7500024C0C5010197F1F70894E11CF11C011DCB
:10E76000111D21E2E2162EE4F20620E0020720E06D
:10E77000120718F031E0C32ED12CC801B70127ECE5
:10E780003BE140E050E00F9441FE611571058105C9
:10E79000910519F485B1805885B98091C00087FD35
:10E7A00003C0C114D104A9F2A6014F5F5F4FC25E3E
:10E7B000DE4F59834883CE51D140C25EDE4F8881FF
:10E7C0009981CE51D140019711F00D9410FEC05D9A
:10E7D000DE4F19821882C053D14060E0C15DDE4F28
:10E7E0001882CF52D14088249924C35DDE4F19820C
:10E7F0001882CD52D140C05EDE4F188219821A8233
:10E800001B82C052D140CE5CDE4F188219821A8220
:10E810001B82C253D140EE24FF2487010BBFF701B6
:10E8200007911691C45CDE4F19830883CC53D14005
:10E830000D940BFEC25EDE4F28813981CE51D1404E
:10E840002130310509F52091C600C25EDE4F1982E4
:10E850001882CE51D14022C02F5F3F4F4F4F5F4FA4
:10E86000213082E138078AE7480780E0580780F0C6
:10E87000C45CDE4FE881F981CC53D140EF5FFF4F9C
:10E8800019F0EE27FF27099420E030E040E050E047
:10E890008091C00087FFE0CF2091C600C35DDE4FAE
:10E8A00048815981CD52D1404F5F5F4FC35DDE4FEC
:10E8B00059834883CD52D140213209F063C64A3092
:10E8C000510508F05FC60894811C911C53E0851621
:10E8D000910409F059C600E010E018C081E280936D
:10E8E000C6008091C00086FFFCCF8091C00080648C
:10E8F0008093C0002F5F3F4F2931310579F70F9486
:10E90000DCF10F5F1F4F0530110519F020E030E0FA
:10E91000E5CF10920A0210920B0210920C02109294
:10E920000D02109206021092070210920802109235
:10E930000902109202021092030210920402109235
:10E9400005028FEE90EE60E00F94F5F180E191EE1C
:10E9500060E00F94C2F18091C00087FFFCCF9091DE
:10E96000C600903608F09F759032B8F09093C600BC
:10E970008091C00086FFFCCF8091C00080648093AE
:10E98000C000A0E2A093C6008091C00086FFFCCF2B
:10E990008091C00080648093C000983409F4D7C18E
:10E9A0009934B8F4923409F459C1933458F490333B
:10E9B00019F1903308F4E3C59F33A1F1903409F0C5
:10E9C000DEC5BDC0953409F470C1963409F0D7C5D1
:10E9D00098C1923509F42BC2933538F49C3409F46C
:10E9E000F5C1913509F0CBC518C2963509F445C279
:10E9F000993509F0C4C567C483E792EE62E00F94CD
:10EA0000F5F110920602109207021092080210927D
:10EA1000090210920A0210920B0210920C0210923C
:10EA20000D0213C18FE792EE62E00F94F5F18FEEC5
:10EA300090EE60E00F94F5F181E291EE60E00F94CA
:10EA4000C2F187EB91EE60E00F94F5F180E391EE77
:10EA500060E00F94C2F184EE90EE60E00F94F5F167
:10EA60008FE391EE60E00F94C2F186E090E061E008
:10EA700070E00F9434F20F94DCF18DE591EE60E0DC
:10EA80000F94C2F189EC91EE60E00F94F5F18EE401
:10EA900091EE60E00F94C2F183EC91EE60E00F9490
:10EAA000F5F18CE691EE60E00F94C2F18EE10F94E7
:10EAB0000DF288E90F940DF281E00F940DF20F949E
:10EAC000DCF18BE791EE60E00F94C2F119E0E0E039
:10EAD000F0E010935700E4918E2F0F940DF20F94F5
:10EAE000DCF18AE891EE60E00F94C2F1E3E0F0E03F
:10EAF00010935700E4918E2F0F940DF20F94DCF1D8
:10EB000089E991EE60E00F94C2F1E2E0F0E0109349
:10EB10005700E4918E2F0F940DF20F94DCF188EAE8
:10EB200091EE60E00F94C2F1E1E0F0E01093570045
:10EB30001491812F0F940DF20F94DCF107CF8BE825
:10EB400092EE62E00F94F5F18BE492EE60E00F94A8
:10EB5000F5F10F94DCF100E010E019C0C8016F2D51
:10EB60000F947FFEFF2031F489E492EE60E00F9471
:10EB7000C2F10BC0F092C6008091C00086FFFCCFAE
:10EB80008091C00080648093C0000F5F1F4FC80158
:10EB900081519F41A0E0B0E0ABBFFC01F790BAE229
:10EBA000FB1621F0E2E000301E07C1F60F94DCF105
:10EBB0000F94DCF187E592EE60E00F94F5F10F948D
:10EBC000DCF1CC24DD2400E010E01EC0C8010F946D
:10EBD00077FEF82E882331F489E492EE60E00F94FA
:10EBE000C2F10BC08093C6008091C00086FFFCCFAD
:10EBF0008091C00080648093C000FE1419F00894D6
:10EC0000C11CD11C0F5F1F4FC80181519F41A0E063
:10EC1000B0E0ABBFFC01E790FAE2EF1621F022E092
:10EC20000030120799F60F94DCF10F94DCF182E6C4
:10EC300092EE60E00F94C2F1C60161E070E00F94C3
:10EC400034F20F94DCF10F94DCF110920202109276
:10EC50000302109204021092050278CE89E992EE26
:10EC600062E00F94F5F1279A2F9A16C02F9880E052
:10EC700090E0E0EDF7E03197F1F7019684369105E9
:10EC8000C1F72F9A80E090E0E0EDF7E03197F1F7DF
:10EC9000019684369105C1F78091C00087FFE6CFC9
:10ECA0008091C00087FFFCCF64C485EA92EE62E0E9
:10ECB0000F94F5F140910202509103026091040219
:10ECC0007091050281E020E10F9491F2809102029F
:10ECD00090910302A0910402B091050280509F4FD1
:10ECE000AF4FBF4F8093020290930302A0930402A0
:10ECF000B093050280509041A040B04008F426CE69
:10ED0000A4CF83EB92EE62E00F94F5F140910602FE
:10ED100050910702609108027091090280E020E1A1
:10ED20000F9491F28091060290910702A09108023F
:10ED3000B091090280509F4FAF4FBF4F80930602A2
:10ED400090930702A0930802B0930902FFCD80ECD4
:10ED500092EE62E00F94F5F183E792EE60E00F949B
:10ED6000F5F18FE792EE60E00F94F5F18BE892EE0B
:10ED700060E00F94F5F189E992EE60E00F94F5F10F
:10ED800085EA92EE60E00F94F5F183EB92EE60E09D
:10ED90000F94F5F180EC92EE60E00F94F5F187ECC2
:10EDA00092EE60E00F94F5F188ED92EE60E00F9442
:10EDB000F5F18FED92EE60E00F94F5F18AEE92EEB0
:10EDC00060E00F94F5F183E093EEBDCD87EC92EE19
:10EDD00062E00F94F5F181E40F947BF282E40F94EA
:10EDE0007BF283E40F947BF284E40F947BF285E45E
:10EDF0000F947BF286E40F947BF287E40F947BF20E
:10EE000088E40F947BF28AE40F947BF28BE40F94F6
:10EE10007BF28CE40F947BF299CD88ED92EE62E068
:10EE20000F94F5F1772473948824992409C48FED05
:10EE300092EE62E00F94F5F140910A0250910B02BC
:10EE400060910C0270910D0282E020E10F9491F22A
:10EE500080910A0290910B02A0910C02B0910D02D8
:10EE600080509F4FAF4FBF4F80930A0290930B0289
:10EE7000A0930C02B0930D0269CD8AEE92EE62E08F
:10EE80000F94F5F184EE90EE60E00F94F5F18FECC5
:10EE900091EE60E00F94F5F1662477244301CC5D98
:10EEA000DE4F19821882C452D140D401C301B695F5
:10EEB000A79597958795CA5DDE4F88839983AA8326
:10EEC000BB83C652D140CC5DDE4FA881B981C4520C
:10EED000D1401196CC5DDE4FB983A883C452D14096
:10EEE000CD0162E070E00F9434F2B0E2B093C6005E
:10EEF0008091C00086FFFCCF8091C0008064809329
:10EF0000C000EDE2E093C6008091C00086FFFCCF18
:10EF10008091C00080648093C000F0E2F093C6004E
:10EF20008091C00086FFFCCF8091C00080648093F8
:10EF3000C000CA5DDE4FE880F9800A811B81C6529D
:10EF4000D140BB27A12F902F8F2D0F940DF2CA5DBA
:10EF5000DE4F8881C652D1400F940DF2B0E2FB2EF5
:10EF6000F092C6008091C00086FFFCCF8091C00067
:10EF700080648093C0000DE30093C6008091C000C0
:10EF800086FFFCCF8091C00080648093C00010E2B7
:10EF90001093C6008091C00086FFFCCF8091C00016
:10EFA00080648093C0008BBEF3012791C65DDE4F65
:10EFB0002883CA52D140A22EBB24CC24DD2408943D
:10EFC000611C711C811C911C8BBEF3018791282E42
:10EFD0003324442455240894611C711C811C911C09
:10EFE0008BBEF3013791C55DDE4F3883CB52D140E4
:10EFF0000894611C711C811C911C8BBEF30147910C
:10F00000C45DDE4F4883CC52D140ADEFEA2EAFEF66
:10F01000FA2EAFEF0A2FAFEF1A2F6E0C7F1C801E57
:10F02000911E142D032DF22CEE24EA0CFB1C0C1D5A
:10F030001D1D0F940DF220E22093C6008091C000A8
:10F0400086FFFCCF8091C00080648093C000C65DC5
:10F05000DE4F8881CA52D1400F940DF230E23093D6
:10F06000C6008091C00086FFFCCF8091C000806404
:10F070008093C000C45DDE4F8881CC52D1400F9494
:10F080000DF240E24093C6008091C00086FFFCCFA5
:10F090008091C00080648093C000C55DDE4F888190
:10F0A000CB52D1400F940DF250E25093C6008091A4
:10F0B000C00086FFFCCF8091C00080648093C000B8
:10F0C0008FEFE8168FEFF80680E0080780E018075A
:10F0D00031F484E092EE60E00F94C2F1DFC0D80119
:10F0E000C7018070907CA070B0708050904CA040A0
:10F0F000B040D1F52FEF3FE340E050E0E222F322B1
:10F1000004231523CA5DDE4FA880B980CA80DB8046
:10F11000C652D140AE0CBF1CC01ED11EAA0CBB1CD7
:10F12000CC1CDD1C8EE092EE60E00F94C2F1BB2798
:10F13000A12F902F8F2D0F940DF28E2D0F940DF285
:10F1400030E23093C6008091C00086FFFCCF8091F2
:10F15000C00080648093C0004EE34093C60080915D
:10F16000C00086FFFCCF87C08EE09EEFA0E0B0E03D
:10F17000E822F9220A231B239CE0E91694E9F90608
:10F1800090E0090790E0190709F088C0C45DDE4FE0
:10F19000A881CC52D140EA2EFF2400E010E0102FCD
:10F1A0000F2DFE2CEE24C55DDE4FB881CB52D14031
:10F1B000EB0EF11C011D111DD601C501817090706F
:10F1C000A070B070DC0199278827E80EF91E0A1F8D
:10F1D0001B1F20EF30E040E050E0A222B322C42207
:10F1E000D52241E1AA0CBB1CCC1CDD1C4A95D1F7F1
:10F1F000EA0CFB1C0C1D1D1D81E090E0A0E0B0E0BE
:10F20000282239224A225B2235E1220C331C441C7D
:10F21000551C3A95D1F7E20CF31C041D151D57013E
:10F220006801AA0CBB1CCC1CDD1C85E192EE60E0E1
:10F230000F94C2F1C801AA27BB270F940DF2BB2778
:10F24000A12F902F8F2D0F940DF28E2D0F940DF274
:10F2500090E29093C6008091C00086FFFCCF809121
:10F26000C00080648093C000AEE3A093C60080918C
:10F27000C00086FFFCCF8091C00080648093C000F6
:10F28000C601AA27BB270F940DF2BB27AD2D9C2DDD
:10F290008B2D0F940DF28A2D0F940DF20F94DCF14B
:10F2A000CC5DDE4FE881F981C452D140F99709F471
:10F2B0004DCBF4E0EF2EF12C012D112D6E0C7F1CA7
:10F2C000801E911EF2CD83E093EE62E00F94F5F183
:10F2D0008AE192EE60E00F94C2F18091C00087FF56
:10F2E000FCCF1091C6001F751093C6008091C0001E
:10F2F00086FFFCCF8091C00080648093C0000F9493
:10F30000DCF1812F81548A3108F036C1163409F4BA
:10F3100095C0173490F4133409F44EC0143430F40B
:10F320001134F1F0123409F01DC130C0143409F465
:10F3300059C0153409F016C16BC01A3409F4C4C0A1
:10F340001B3438F4173409F48FC0183409F00AC19B
:10F35000A1C01B3409F4D2C01C3409F003C1E8C0B9
:10F360008FEF81B90DC082B1809582B980E090E0C5
:10F37000E0EDF7E03197F1F70196883C9105C1F790
:10F380008091C00087FFEFCF12B8EFC08FEF84B934
:10F390000DC085B1809585B980E090E0E0EDF7E0A3
:10F3A0003197F1F70196883C9105C1F78091C00033
:10F3B00087FFEFCF15B8D9C08FEF87B90DC088B1DF
:10F3C000809588B980E090E0E0EDF7E03197F1F7C3
:10F3D0000196883C9105C1F78091C00087FFEFCF6F
:10F3E00018B8C3C08FEF8AB90DC08BB180958BB9A7
:10F3F00080E090E0E0EDF7E03197F1F70196883C8E
:10F400009105C1F78091C00087FFEFCF1BB8ADC059
:10F410008FEF8DB90DC08EB180958EB980E090E0F0
:10F42000E0EDF7E03197F1F70196883C9105C1F7DF
:10F430008091C00087FFEFCF1EB897C08FEF80BBD1
:10F440000DC081B3809581BB80E090E0E0EDF7E0F6
:10F450003197F1F70196883C9105C1F78091C00082
:10F4600087FFEFCF11BA81C08FEF83BB0DC084B38C
:10F47000809584BB80E090E0E0EDF7E03197F1F714
:10F480000196883C9105C1F78091C00087FFEFCFBE
:10F4900014BA6BC08FEF809301010FC080910201FD
:10F4A00080958093020180E090E0E0EDF7E03197F5
:10F4B000F1F70196883C9105C1F78091C00087FF64
:10F4C000EDCF1092020151C08FEF809304010FC065
:10F4D0008091050180958093050180E090E0E0ED4A
:10F4E000F7E03197F1F70196883C9105C1F78091DB
:10F4F000C00087FFEDCF1092050137C08FEF8093DA
:10F5000007010FC08091080180958093080180E079
:10F5100090E0E0EDF7E03197F1F70196883C910536
:10F52000C1F78091C00087FFEDCF109208011DC088
:10F530008FEF80930A010FC080910B01809580931B
:10F540000B0180E090E0E0EDF7E03197F1F70196F4
:10F55000883C9105C1F78091C00087FFEDCF1092E4
:10F560000B0103C085E292EEEEC98091C00087FFD7
:10F57000FCCF8091C600EAC988E392EEE4C98CE131
:10F5800091EEE1C988249924933011F1943028F444
:10F59000913089F09230B8F408C0953061F195301F
:10F5A000F0F0963009F048C043C02B3109F042C951
:10F5B00091E06BE13FC96227C15DDE4F2883CF52E6
:10F5C000D14092E037C9B22FA0E0622793E032C960
:10F5D000822F90E0A82BB92B622794E02BC92E3004
:10F5E00009F039C3622795E0C05DDE4F19821882A9
:10F5F000C053D1401FC9E1E0F0E0EC0FFD1FC05D3A
:10F60000DE4F08811981C053D140E00FF11F2083E4
:10F610000F5F1F4FC05DDE4F19830883C053D14079
:10F6200062270A171B0709F005C9D80196E002C92D
:10F63000261709F010C303C0973009F0FBC87724E0
:10F640009981933109F412C19431C8F4963009F4C8
:10F65000D8C0973050F4923009F406C1933009F4C1
:10F660006DC0913009F059C253C0913109F477C08F
:10F67000923108F0BBC0903109F04FC2F5C098310B
:10F6800009F487C0993150F4953109F4EFC09531F0
:10F6900008F4C6C1963109F040C2C2C19A3109F4DA
:10F6A0006CC09A3108F491C09B3109F45BC09D3164
:10F6B00009F033C29D81903359F48F81882311F46E
:10F6C0009EE11CC0813011F091E018C098E916C08D
:10F6D000892F807591F0903539F4E0E0F0E089E011
:10F6E0008093570094910AC0983539F4E3E0F0E034
:10F6F00089E080935700949101C090E01A821B82A8
:10F700008D818C831D829E831F8227E030E009C299
:10F710001A8288E08B8381E48C8386E58D8382E581
:10F720008E8389E48F8383E5888780E589878FE5E9
:10F730008A8782E38B872BE030E0F3C18A818139AD
:10F7400041F0823941F0803911F48FE005C080E04A
:10F7500003C082E001C08AE01A828B8344C0772410
:10F76000739482C08D81882311F48EE12CC0813086
:10F7700011F081E028C088E926C01A82E1E0F0E0BB
:10F7800089E08093570084918B831C8224E030E0D1
:10F79000C8C18B81803589F48C81883039F4E2E0EE
:10F7A000F0E089E08093570084910DC0E0E0F0E044
:10F7B00089E080935700849106C0E3E0F0E089E09F
:10F7C0008093570084911A82DFCF8D81836C99E0FA
:10F7D000E1E0F0E0082E90935700E89507B600FCB2
:10F7E000FDCF1A821B8223E030E09BC180EC8A832C
:10F7F000CE5CDE4F188219821A821B82C253D1401E
:10F800008EC18A8190E0A0E0B0E0582F44273327D2
:10F8100022278B8190E0A0E0B0E0DC0199278827C7
:10F82000282B392B4A2B5B2B8D8190E0A0E0B0E098
:10F83000282B392B4A2B5B2B8C8190E0A0E0B0E089
:10F84000BA2FA92F982F8827282B392B4A2B5B2BCF
:10F85000220F331F441F551FC05EDE4F288339839C
:10F860004A835B83C052D1401A8259C13A81C95C34
:10F87000DE4F3883C753D140CA5CDE4F1882C6536F
:10F88000D1408B81C82EDD24CA5CDE4F488159816E
:10F89000C653D140C42AD52A933109F082C0CE5C28
:10F8A000DE4F88819981AA81BB81C253D1408050AB
:10F8B000904CA340B04030F583E0CE5CDE4FE88052
:10F8C000F9800A811B81C253D140F70100935B008C
:10F8D00080935700E89507B600FCFDCFCE5CDE4F65
:10F8E000088119812A813B81C253D14000501F4FAA
:10F8F0002F4F3F4FCE5CDE4F088319832A833B8313
:10F90000C253D140C05EDE4F488159816A817B81FC
:10F91000C052D140DE011B9631E08C9111962C91A2
:10F9200011971296C75CDE4F2883C953D140C85C3B
:10F93000DE4F1882C853D14090E0C85CDE4FE881AA
:10F94000F981C853D1408E2B9F2B0C01FA01609393
:10F950005B0030935700E89511244E5F5F4F6F4F67
:10F960007F4F0EEFE02E0FEFF02ECE0CDF1CC114F8
:10F97000D10499F685E0C05EDE4F088119812A81A5
:10F980003B81C052D140F80120935B008093570027
:10F99000E89507B600FCFDCF81E180935700E8951C
:10F9A00035C0C05EDE4F88819981AA81BB81C0527B
:10F9B000D140B695A795979587957C018601ABE0D8
:10F9C000AA2EB12CAC0EBD1E0BC0D5016D915D01F0
:10F9D000C7010F947FFE0894E11CF11C01501040F8
:10F9E0000115110591F7A60160E070E0440F551F65
:10F9F000661F771FC05EDE4FE880F9800A811B8199
:10FA0000C052D1404E0D5F1D601F711F1A82C05E33
:10FA1000DE4F488359836A837B83C052D1407FC0C5
:10FA2000FA80C55CDE4FF882CB53D140C65CDE4F16
:10FA30001882CA53D1408B81C82EDD24C65CDE4FAC
:10FA400008811981CA53D140C02AD12A1A828981DA
:10FA5000BE016D5F7F4F843121F59601C05EDE4FA0
:10FA6000E880F9800A811B81C052D1400BBFF701A9
:10FA700087919691DB018C9311969C936E5F7F4FDB
:10FA8000D801C7010296A11DB11DC05EDE4F88835B
:10FA90009983AA83BB83C052D14022503040F1F6F3
:10FAA00036C0C05EDE4F288139814A815B81C052F9
:10FAB000D1400894C108D108760100E010E0089414
:10FAC000C11CD11C0894E11CF11C011D111DE20E8A
:10FAD000F31E041F151F21BDBB27A52F942F832FB5
:10FAE00082BD2F5F3F4F4F4F5F4FF89A80B5DB01CC
:10FAF0008D93BD012E153F054007510761F7C05E8C
:10FB0000DE4F288339834A835B83C052D1409601FC
:10FB10002D5F3F4FFB01108204C080EC8A8322E0FE
:10FB200030E08BE18093C6008091C00086FFFCCF5F
:10FB30008091C00080648093C000C15DDE4FF88179
:10FB4000CF52D140F093C6008091C00086FFFCCF19
:10FB50008091C00080648093C000432F3093C60022
:10FB60008091C00086FFFCCF8091C00080648093AC
:10FB7000C000922F2093C6008091C00086FFFCCF6A
:10FB80008091C00080648093C0008EE08093C600A6
:10FB90008091C00086FFFCCF8091C000806480937C
:10FBA000C00065E1C15DDE4FE880CF52D1406E25D7
:10FBB00069276427FE01319610C090819093C6009A
:10FBC0008091C00086FFFCCF31968091C000806498
:10FBD0008093C0006927215030402115310569F715
:10FBE0006093C6008091C00086FFFCCF8091C0006A
:10FBF00080648093C00085B1805885B9772081F4F6
:10FC0000C15DDE4F0881CF52D1400F5FC15DDE4F35
:10FC10000883CF52D14090E0A0E0B0E00D941AF4F8
:10FC200027982F9880E090E020ED37E0F901319798
:10FC3000F1F7019684369105C9F700008091C00064
:10FC40008D7F8093C00081E180935700E895EE2777
:10FC5000FF270994FFCF90E00D941AF497FB092E2B
:10FC600007260AD077FD04D02ED006D000201AF443
:10FC7000709561957F4F0895F6F7909581959F4F08
:10FC80000895A1E21A2EAA1BBB1BFD010DC0AA1FDD
:10FC9000BB1FEE1FFF1FA217B307E407F50720F0F5
:10FCA000A21BB30BE40BF50B661F771F881F991F70
:10FCB0001A9469F760957095809590959B01AC01B9
:10FCC000BD01CF010895AA1BBB1B51E107C0AA1FAC
:10FCD000BB1FA617B70710F0A61BB70B881F991FED
:10FCE0005A95A9F780959095BC01CD010895F99991
:10FCF000FECF92BD81BDF89A992780B50895262F31
:10FD0000F999FECF1FBA92BD81BD20BD0FB6F89400
:0EFD1000FA9AF99A0FBE01960895F894FFCF63
:00000001FF
